:0A00060000308A001C28000034308E
:100010008400000803191B280130F800F701F70BD2
:100020000F28F80B0E284A30F700F70B15280000B0
:100030000000800B0C28003484011F3083058316D8
:100040001F08C0399F009B01073083129F001E309C
:1000500083168500F03086008312850186018316A1
:1000600081130030831285180130013C031D3B28A9
:10007000831631288312061086100030861B01304B
:10008000013C03193B28861506148610F030B40095
:10009000072006148614003005190130003A0319B0
:1000A0005F280830B300FA30B4000720B30B5328A0
:1000B00086140610B430B400072086113B280030A7
:0E00C000861B0130003A031958285F286300A0
:040000008A01032846
:00000001FF
